:020000040000FA
:10000000F86A7D0EF76EC00EF66EA68EA69CA684CC
:10001000A688F29E550EA76EAA0EA76EA6820000B5
:10002000F28E010EF56E0D00EF0EF56E0D00300E26
:10003000F56E0D00F00EF56EF56A0D000D000D0069
:100040000C00A68EA69CA684A698F29E550EA76EBE
:10005000AA0EA76EA6820000F28EA6948E0EC16E26
:10006000E10E926E100E806E8082FFD701EF30F0AD
:10600000FFD7E0CF0AF50501F2AE03D0F29E128F62
:1060100001D0129FE8CF00F5D8CF01F5EACF02F505
:10602000E9CF03F5E2CF04F5E1CF05F5DACF06F5C8
:10603000D9CF07F5FBCF08F5FACF09F5F8CF0BF567
:10604000F7CF0CF5F6CF0DF5D5AE03D0D59E128166
:1060500001D01291CDA003D0CD90128301D0129324
:10606000CAA403D0CA94128501D01295B1A003D05E
:10607000B190128701D01297D49C2CEC31F059B515
:1060800001D0396BC5EC30F05851130B130A20E0E6
:1060900059B506D0596BD9EC36F07CEC35F001D00F
:1060A0005995126B0E6B0F6B106B116B58B310D0B0
:1060B000700EF76EBA0EF66E0CEC31F0700EF76ED5
:1060C000E00EF66E0CEC31F034EC31F0BDEC31F05A
:1060D00058AB2CD0D4AA05D010C50EF511C50FF5BC
:1060E00025D058AF1AD0A0EC31F039B901D039839E
:1060F000FECF10F5FDCF11F5AB9EAB8E510E9EA8D5
:10610000FED7AD6E210E9EA8FED7AD6E3E0E9EA8A8
:10611000FED7AD6EBDEC31F009D0D488B8500E6F0B
:10612000B7500F6FD498D8900F370E37FECF10F5B9
:10613000FDCF11F558AB1AD0589B58AF0AD0D4BA3E
:1061400008D09EAA06D0710EF76E920EF66E0CEC79
:1061500031F058AD09D0589DE6EC36F0710EF76E6F
:10616000980EF66E0CEC31F02DEC37F0710EF76EE8
:10617000920EF66E0CEC31F0598167EC32F05991C9
:106180000AEC33F0BDEC31F0F1D7FCAC07D0FC9C4D
:10619000740EF76E8C0EF66E0CEC31F0FCAE07D080
:1061A000FC9E740EF76E7A0EF66E0CEC31F0D05049
:1061B0001F0B1F0A0DE158AB0AD058AF07D0D4BA55
:1061C00005D0C6EC32F09EBA01D0D09201D0D09268
:1061D000D0B206D0DD0E586F596BD082D08001D07E
:1061E0005883D0B009D05891D080740EF76E5E0EEF
:1061F000F66E0CEC31F001D05881D0B80BD0589924
:10620000D08859B506D0740EF76E120EF66E0CECEF
:1062100031F001D0588912000800F55014EC31F02B
:106220000B00F550FBE112007F0B9EA8FED7AD6E70
:106230001200ABA202D0AB98AB889EAAFED7AE509C
:106240009EAA02D0AB9EAB8E12000D0E14EC31F064
:106250000A0E14EC31F012001E0EAF6EAC84AC8A44
:10626000AC98AB88AB8E1200A0EC31F039B949D0B4
:106270009EAA05D0AE50AB9EAB8E9EBAFBD7020E47
:10628000136F1353D8B431D0730EF76E360EF66E0B
:106290000CEC31F0730EF76E5A0EF66E0CEC31F01A
:1062A0005B0E14EC31F0200E14EC31F0132FFBD701
:1062B0005D0E14EC31F0030E136F080E14EC31F088
:1062C000132FFBD7020E136FABA202D0AB98AB8893
:1062D0009EBA15D0640E146FC6EC32F01407FCE1C0
:1062E000230E14EC31F0132FEFD725EC31F0710EA3
:1062F000F76E920EF66E0CEC31F0398102D025EC7F
:1063000031F012003989000EF76E000EF66E030EA2
:10631000156F0900F55207E00900F550EF0801E19B
:1063200039990DD00AD00900F550EF0803E13999E9
:1063300006D003D0F55001E002D01507EAE11200C3
:106340003989F76AF66A600E616F000E626F0900A4
:10635000F550FF0A01E009D0620701E261076253CC
:1063600003E1615301E101D0F2D7615304E16253CB
:1063700001E0399901D03999120039AD09D0D7EC33
:1063800033F0720EF76E1E0EF66E0CEC31F01DD06F
:1063900039AF09D0D7EC33F0720EF76E3C0EF66EC3
:1063A0000CEC31F012D039A907D0720EF76E640EE2
:1063B000F66E0CEC31F009D039A303D0E7EC31F0E4
:1063C00004D039A102D023EC32F0396B1200060060
:1063D00006005851130B130A07E0FC2A000EFF6E4B
:1063E000000EFE6E000EFD6E588BD48AD48C12A166
:1063F00001D0D58E12A301D0CD8012A501D0CA84C0
:1064000012A701D0B18012AF01D0F28E0BC5F8FFF8
:106410000CC5F7FF0DC5F6FF0AC5E0FF09C5FAFF79
:1064200008C5FBFF02C5EAFF03C5E9FF04C5E2FF9B
:1064300005C5E1FF06C5DAFF07C5D9FF01C5D8FFCD
:1064400000C5E8FFE1000600060058AF06D0710E57
:10645000F76EF20EF66E0CEC31F05851130B130A76
:1064600007E0FC2A000EFF6E000EFE6E000EFD6EB1
:10647000588BD49AD48C12A101D0D58E12A301D0FE
:10648000CD8012A501D0CA8412A701D0B18012AF6D
:1064900001D0F28E0BC5F8FF0CC5F7FF0DC5F6FF56
:1064A0000AC5E0FF09C5FAFF08C5FBFF02C5EAFF00
:1064B00003C5E9FF04C5E2FF05C5E1FF06C5DAFF34
:1064C00007C5D9FF01C5D8FF00C5E8FFE100AB9EB5
:1064D000AB8E05EE19F00C0E166F186B19EC31F03F
:1064E000EF6E59A105D0CEEC32F0185301E02CD05C
:1064F000EF50FDEC32F0185303E0598325D001D062
:106500005993EF500D0A04E1000EEF6E9EDE1CD091
:10651000EF50080A0FE1190EE9180BE0080E14EC11
:1065200031F0200E14EC31F0080E14EC31F0ED5285
:10653000162B08D0EE5014EC31F0160703E1000ED4
:10654000EF6E83DE1653CAE11200186B310A03E1C5
:106550000A0E186F04D0030A02E1140E186F19EC2A
:1065600031F0185310E00F0B18270A0E185F730E46
:10657000F76E740EF66E1851D890F62601E3F72ADE
:106580000800F5CF18F519EC31F01200E86A200E7A
:10659000156FE806FEE11507FCE112002009136FF4
:1065A000680A02E1010E186F1351740A02E1020E2B
:1065B000186F13516C0A02E1030E186F1351640A2D
:1065C00002E1040E186F1351620A02E1050E186F02
:1065D0001351770A02E1060E186F1351720A02E195
:1065E000070E186F1351730A02E1080E186F13514A
:1065F0006D0A02E1090E186F12001B0A0AE119EC7C
:1066000031F0EF6E5B0A05E119EC31F0EF6EA5ECAD
:1066100032F01200185302E010EC33F0196B120044
:10662000FB6A660EFA6ED8901837D89018373C0E71
:10663000D890182501E3FA2A1851F9260000000025
:1066400038EF33F03FEF33F043EF33F04EEF33F0FA
:1066500059EF33F05CEF33F063EF33F069EF33F071
:106660006FEF33F072EF33F079EF33F080EF33F008
:10667000700EF76EE00EF66E0CEC31F01200589DC5
:10668000589BFF001200588D92D8A2D85985280E29
:10669000146FC6EC32F01407FCE1FF00E6EC36F0B4
:1066A000710EF76E980EF66E0CEC31F02DEC37F0A3
:1066B000120018EC35F01200720EF76EA20EF66E94
:1066C000ABDD64DA1200A0EC31F039B901D03981C8
:1066D0001200A0EC31F039B901D039831200F1EC8D
:1066E00037F01200740EF76E260EF66E0CEC31F0D9
:1066F0001200740EF76E2E0EF66E0CEC31F01200D6
:10670000740EF76E360EF66E0CEC31F089EC33F049
:10671000120067EC32F0050EEA6E190EE96E740E87
:10672000F76EEC0EF66E0CEC31F0000EF86E31ECFC
:1067300038F037C5F7FF000EF66EFF0E156F100E1E
:10674000166F100E161911E1F850C7EC37F0200E35
:1067500014EC31F0F750C7EC37F0F63820EC38F095
:1067600014EC31F0200E14EC31F00900F6A003D047
:10677000F5CF14F506D0F550C7EC37F01451C7EC3F
:1067800037F0F6B003D0200E14EC31F01607000EEF
:10679000161908E10D0E14EC31F00A0E14EC31F06C
:1067A000100E166F1507CDE125EC31F01200000E2A
:1067B000F86EF76EF66E21EE80F02AD9400EF626BE
:1067C000D8B0F72ADD52D952F8E1DA52F6E11200D8
:1067D000396B2CEC31F0710EF76EC00EF66E0CECCE
:1067E00031F019EC31F03A0AD8A4FBD7326B25EC22
:1067F00034F01F0B316FD890313325EC34F0336F08
:1068000025EC34F0346F25EC34F0356F010AD8B440
:106810000BD03551020AD8B409D037EC34F039BF67
:1068200013D039BD11D0DDD725EC34F0A0EC31F018
:1068300039B90AD0720EF76E000EF66E0CEC31F01C
:1068400019EC31F0D9EC34F0120019EC31F0BF0F33
:10685000D8A0070F0A0F376F373B19EC31F0BF0F85
:10686000D8A0070F0A0F371337513227120005EE51
:1068700019F031C516F525EC34F0EE6E25EC34F048
:10688000EE6E162FF8D725EC34F03253D8B402D080
:10689000398D15D03551040AD8B407D03551D8A454
:1068A0000ED075D839AF0FD80AD01A51300AD8A4F3
:1068B00006D019EC31F03A0AD8A4FBD700D02E0E3E
:1068C00014EC31F01200000EF86E33C5F7FFF80E2D
:1068D0003415F66E050EEA6E290EE96E040E166F7B
:1068E000FEEC34F0070E3415146F290E1425E96EF2
:1068F000050EEA6E050EE26E190EE16ED8901433A5
:1069000031C516F5E6CFEEFFE6CFEEFF142B1607E6
:10691000D8B404D01451040AD8A4F4D7000EF86EE9
:1069200033C5F7FFF80E3415F66E050EEA6E290E24
:10693000E96EEBEC34F01653D8B4C1D70900050E5C
:10694000EA6E290EE96E16C514F5040E166FFEECFC
:1069500034F014C516F5050EEA6E290EE96EE6CF81
:10696000EEFFE6CFEEFF162FAFEF34F0050EEA6E26
:10697000290EE96EF86A33C5F7FFF80E3415F66E86
:10698000080EF626D8B0F72AEBEC34F0120033C527
:106990005EF534C55FF531C560F5399F600E335D36
:1069A00007E605E1000E345D01E6398F01D0398F2D
:1069B0001200740EF76ECC0EF66E0CEC31F05E51D8
:1069C000C7EC37F0D8906035FE0F5F25C7EC37F085
:1069D00025EC31F01200040E146F0A00EECFF5FF23
:1069E0000F00EECFF5FF0F00142FEEEF34F0A68E60
:1069F000A69CA6840FEC35F0A69412000900F5CFF2
:106A0000EEFF0900F5CFEEFF162FFEEF34F0120077
:106A1000A68EA69CA684A6880FEC35F01200D4AEF4
:106A200006D0550EA76EAA0EA76EA6820000120011
:106A3000730EF76EC20EF66E0CEC31F0730EF76E3D
:106A4000840EF66E0CEC31F067EC32F005EE19F0C6
:106A500059B348D0EF5244E0EE52EF521EE1ED52EE
:106A6000EF502009720A0AE17CEC35F0730EF76EE4
:106A7000A60EF66E0CEC31F03ED00ED0EF50200991
:106A8000640A04E19EEC35F036D006D0740EF76E41
:106A90009E0EF66E0CEC31F022D0ED52040E156F06
:106AA0005A8D5AAD03D0EE50C9EC36F01507F9E116
:106AB0005AAD0FD0EF5206E187EC35F09EEC35F081
:106AC0001AD006D0740EF76E9E0EF66E0CEC31F0F6
:106AD00006D0740EF76E9E0EF66E0CEC31F001D0FF
:106AE0000AD008D025EC31F0740EF76E9E0EF66ECB
:106AF0000CEC31F0A3D71200588D588FD4880F0EAC
:106B0000B912FF0EB86EFF0EB76ED4981200588DF2
:106B1000589F05EE19F01FEEB8F0D488F00EB916A4
:106B2000020E156F31EC38F037C5E5FFEE50150752
:106B3000F9E1D890B832B732D4981200D4880F0E49
:106B4000B9140F0A1BE0730EF76E940EF66E0CEC80
:106B500031F0300E14EC31F0780E14EC31F0D890A6
:106B6000B736B836B850C7EC37F0B750C7EC37F087
:106B7000D890B832B73225EC31F006D0730EF76EEC
:106B8000A60EF66E0CEC31F0D4981200730EF76E70
:106B9000300EF66E0CEC31F067EC32F059B315D0D4
:106BA00005EE19F0EF520FE032EC36F05ABF04D088
:106BB000EFEC35F013D006D0740EF76E9E0EF66E25
:106BC0000CEC31F001D00AD008D025EC31F0740E75
:106BD000F76E9E0EF66E0CEC31F0D8D712000A0E4E
:106BE000156F15EE3AF0E7AE07D05DC5E6FF5CC560
:106BF000E6FF5BC5E7FF35D0E4505C1925E1E450C2
:106C00005B1921E15D531AE1E552E552E2CFEAFF5B
:106C1000E1CFE9FFEE52EE52EE52150702E1E78EA8
:106C20000CD0EFBE07D0EECFE6FFEECFE6FFEECF03
:106C3000E6FF02D0E78E01D0F0D704D0E552E5524E
:106C40005DC5E7FF0ED001D0E652150708E1740ECE
:106C5000F76EB40EF66E0CEC31F003D001D0E652B4
:106C6000C2D712005A6B5B6B5C6B5D6B05EE19F063
:106C7000030E156F5A8D5B390F0B5C6F5B39F00B90
:106C80005B6FEF503AEC38F05B135AAD03D0EE5027
:106C9000C9EC36F01507EFE15AAD07D0060E5C5D82
:106CA00004E65C510F0A01E05A9D5AAD54D0EF52F0
:106CB00001E150D0EF502009200A47E0EF502009B1
:106CC000610A09E1300E5D1504E1300E300B5D13F1
:106CD00001D05A8F3AD0EF502009620A12E1300EEB
:106CE0005D150DE15D510F0B08E15DBD04D0300E67
:106CF000200B5D1301D05A8F01D05A8F01D05A8FCB
:106D000024D0EF502009680A09E1300E5D1504E136
:106D1000300E100B5D1301D05A8F17D0EF502009A1
:106D20002D0A0CE15DBD08D05D51300B200A02E058
:106D30005D8D01D05A8F01D05A8F07D05D510F0B56
:106D400003E1B5EC36F001D05A8F5AAF01D002D032
:106D5000EC52ADE101D05A8F5ABF06D05D510F0BF6
:106D600003E15DAD01D05A8F1200EF5020093108C8
:106D70000EE7090F0AE65D51300B200A02E15A8F37
:106D800003D0EF500F0B5D1301D05A8F01D05A8FF3
:106D900012005A9D2009146F2F080AE70A0F02E615
:106DA0005A8D06D01451600803E7060F01E65A8D8C
:106DB0001200050EE26E3A0EE16E0A0E146F800E9E
:106DC000E66EE66AE66A1407FAE11200730EF76EE1
:106DD000120EF66E0CEC31F001D8120015EE3AF0FE
:106DE0000A0E156FE7AE02D035D02ED0E7CF5DF595
:106DF000E45020EC38F014EC31F0E450C7EC37F0FC
:106E00005DAD02D02D0E01D0200E14EC31F05D519D
:106E1000300B300A08E15D510F0BFB0F02E6020F49
:106E200001D0010E0FD05D51300B200A02E1050E9A
:106E300009D05D510F0BFD0F02E6010F01D0000ECE
:106E4000E846010FEAEC37F0150702E103D001D064
:106E5000E652C8D725EC31F012000E5198D80F51E8
:106E600096D8010EB7D8005192D8010EB3D801A51B
:106E700002D0310E01D0300E14EC31F0200E14ECA3
:106E800031F001A102D0310E01D0300E14EC31F0FE
:106E9000200E14EC31F001A902D0310E01D0300ED9
:106EA00014EC31F0010E96D802516DD803516FD811
:106EB000020E90D8045167D8055169D8020E8AD8BD
:106EC000065161D8075163D8020E84D86BEC37F0B5
:106ED00025EC31F0120015EE3AF00A0E156FE7AE10
:106EE00002D02DD026D0E7CF5DF5E4CFEAFFE4CF86
:106EF000E9FF5D510F0B01E15D2B050E146F5DBDC8
:106F000008D0A0EC37F0EE525D075D510F0BF9E1B0
:106F10000DD05D510F0BFF0FE92601E3EA2AA0EC2B
:106F200037F0ED525D075D510F0BF9E11451EAECBA
:106F300037F0150702E103D001D0E652D0D7120096
:106F40005D51300B300A0AE1EF50DEEC37F014EC03
:106F500031F01451FF0F01E0140714D05D51300BD4
:106F6000200A06E1EF50D1EC37F0010E146F0AD081
:106F7000EF50C7EC37F01451050A02E1030E01D0BF
:106F8000010E146F12005CD814EC31F01200136F74
:106F9000133956D814EC31F0135152D814EC31F0A7
:106FA0001200136F080E166F133702E3310E01D073
:106FB000300E14EC31F01607F7E11200136F810F59
:106FC00002E32A0E06D01351E00F02E22A0E01D08E
:106FD00013511200136F200E14EC31F01307FCE173
:106FE0001200710EF76E340EF66E0CEC31F067EC99
:106FF00032F005EE19F0EF503DD8386FEC5031EC1F
:1070000038F037C536F5EC5003E10BEC38F002D020
:1070100027EC38F01200710EF76E9C0EF66E0CEC39
:1070200031F038C5E2FF36C5E1FFE73809D814EC86
:1070300031F0E75005D814EC31F025EC31F01200B6
:107040000F0BF60F02E23A0F01D0410F120038C5C4
:10705000E2FF36C5E1FFEC5031EC38F037C5E7FF11
:107060001200EF5007D8376F373BEC5003D8371377
:107070003751120020099F0F02E30A0F01D0310F90
:107080001200FC060D0E14EC31F00A0E14EC31F077
:10709000FC50C7EC37F03A0E14EC31F0FE50C7EC60
:1070A00037F0FD50C7EC37F00D0E14EC31F00A0E3E
:1070B00014EC31F0FC2A120061000D0A0909095193
:1070C00077696B42756720666F722050494331388B
:1070D00046343532302076312E300D0A783030008B
:1070E0000D0A463109463209463309463409463508
:1070F0000946360946370946380946390D0A4865B2
:107100006C70097265736554094C6F616409446958
:1071100073706C617909427265616B0957617463C0
:10712000680952756E0953746570094D6F6469661C
:10713000790D0A00446973706C61792F4D6F646931
:10714000667920636F6E74656E7473206F6620526B
:10715000414D206F7220726567697374657220619A
:107160006464726573733A200D0A3C6161613E206C
:10717000746F20446973706C6179202C3C6161618B
:107180002078783E20746F204D6F646966790D0A0F
:10719000000051423E20200051423E00436F6E7479
:1071A000656E74732028486578293A20000045727E
:1071B00061736520436F6D706C6574652E2E2E00B3
:1071C000557365722070726F6772616D206D656DA9
:1071D0006F727920657261736564202D2053656E2E
:1071E00064204845582066696C65206E6F770D0AEB
:1071F000000052756E6E696E672E2E2E0D0A00000D
:107200000D0A446F776E6C6F6164207375636365FC
:10721000737366756C0D0A5C720A783030000D0A63
:107220005472616E736D6974204572726F72202D95
:1072300020436865636B73756D0D0A000D0A577204
:107240006974696E67206F7574736964652055731E
:107250006572204164647265737320537061636565
:107260000D0A00000D0A4E6F207573657220636F62
:10727000646520726573657420766563746F72202F
:107280006973206C6F616465640D0A004E6F205550
:1072900073657220436F6465204C6F616465640D93
:1072A0000A00456E746572207761746368207661A8
:1072B000726961626C652E204578616D706C6573D2
:1072C0003A207C20303132207C2030313220622044
:1072D0007C2030313220612038207C203031322037
:1072E00032207C203031322032202D207C0D0A00CB
:1072F0004D75737420626520616E20416363657310
:10730000732042616E6B20616464726573730D0A51
:10731000000020504320205720205A2043204E2098
:1073200046535230204653523120465352322000A9
:107330002046363E000009095177696B4275672087
:107340004175746F7374617274696E6720557365EB
:107350007220436F64650D0A00000909507265735D
:107360007320616E79206B657920746F2061626F84
:107370007274200000010203040500060708090AD0
:10738000000B0C002046353E2020000020204250FB
:107390003E20200020202020427265616B706F69C2
:1073A0006E74203D2000202020204E6F20627265E8
:1073B000616B706F696E74206973207365740D0A58
:1073C00000003C616161613E20746F207365742030
:1073D000627265616B706F696E742C202752272072
:1073E000746F2072656D6F766520627265616B7077
:1073F0006F696E742C2027442720746F2064697392
:10740000706C617920627265616B706F696E740D6A
:107410000A00526573657420436F6D706C65746506
:107420002E200D0A0000463130200D0A00004631A2
:1074300031200D0A00004631323A456E74657220E3
:1074400048696768204164647265737328322068F4
:10745000657820646967697473293E200000427270
:107460006F776E2D6F757420526573657420446557
:107470007465637465640D0A0000537461636B2066
:107480004F766572666C6F770D0A00005374616306
:107490006B20556E646572666C6F770D0A0020462E
:1074A000363E496E76616C696420436F6D6D616E26
:1074B000640D0A002046363E5761746368204172AD
:1074C0007261792046756C6C0D0A00004869676826
:1074D00065737420416464726573732050726F67C2
:1074E00072616D6D65643A203078000020202020A4
:1074F000202020302031202032203320203420351D
:1075000020203620372020382039202041204220DA
:0C7510002043204420204520460D0A00A6
:020000040030CA
:0300010002181EC4
:02000500830076
:060008000FC00FE00F40E5
:00000001FF
